:020000040030CA
:0E00000000C80F000080800003C003A0034072
:020000040000FA
:020000001FD00F
:020000040000FA
:02000800FFD027
:020000040000FA
:02001800FFD017
:020000040000FA
:10004000CBD09EBA01D0FDD7ABA203D0AB98AB8882
:10005000F8D7EC6EAE50ABA402D0ED50F2D7120040
:10006000ACB201D0FDD7AD6EED5012000500E9DF56
:10007000FD6EED50E6DFFE6EED501200EC6E000EF0
:10008000EFD7A68EA69C88D8F9D7A68EA69C87D82F
:10009000F5D70F0B8DD812000ED0E2D70ED041D07D
:1000A00047D0ECD7FF0019D00DD02CD020D047D0AE
:1000B00033D0E7D7EAD7C5DFE1D7D8DFDFD7C1DF55
:1000C000E8DFFDD7BEDFE46EED50EC6E0900F550C1
:1000D000C7DFE706FAE1E5521200B3DFE46EED5048
:1000E000EC6EDE50BDDFE706FBE1E5521200A9DF52
:1000F000E46EED50A6DFF56E0D00ED50E706FAE177
:10010000E552BCD79EDFE46EED509BDFDE6EED5016
:10011000E706FBE1E552B2D75BD8EC6E0800F528A4
:10012000D2D78FDF8EDFDA6EED50D96EED50A6D7C5
:1001300088DF87DFF76EED50F66EED509FD7EC6EDF
:10014000400EE46EFF0EEC6E0900F550ED14E7066C
:10015000FAE1E55285D7EC6EFD50F66EFE50F76E73
:10016000ED5006001200D96E800AE834DA50DA5AEF
:10017000ED501200F8DFEC6EDE501200F4DFDE6EA0
:10018000ED501200EC6EF29E550EA76EAA0EA76EF1
:10019000A682F28EED501200A684A688F3D7A6841C
:1001A000A6980A00EFDF09001200EF60EF6EED5035
:1001B000E844FD26010BFE22ED50120000EE7FF018
:1001C00010EE8FF08A68EC6E700ED36EED50120058
:1001D000C2DF057069633138000EFC6EEFDFC18A43
:1001E000C18C93889382EC6E330EAF6E240EAC6E8E
:0E01F000900EAB6EED5081A801D061D701D00A
:00000001FF
